:020000040800F2
:10000000880C002085010008410900083909000812
:100010003D0900080D0900089D25000800000000AA
:10002000000000000000000000000000272500087C
:100030001109000800000000C32400082925000859
:100040009F0100089F0100089F0100089F01000810
:100050009F0100089F0100089F0100081509000882
:100060009F0100089F0100089F0100089F010008F0
:100070009F0100089F0100089F0100089F010008E0
:100080009F0100089F0100089F0100089F010008D0
:100090009F0100089F0100089F0100089F010008C0
:1000A0009F0100089F0100089F0100089F010008B0
:1000B0009F0100089F0100089F0100089F010008A0
:1000C0009F0100089F0100089F0100089F01000890
:1000D0009F0100089F0100089F0100089F01000880
:1000E0009F0100089F0100089F0100089F01000870
:1000F0009F0100089F0100089F0100080000000008
:10010000000000009F0100089F010008000000009F
:100110009F0100089F01000800000000000000008F
:100120009F0100089F0100089F0100089F0100082F
:1001300000000000000000000000000000000000BF
:1001400000000000000000000000000000000000AF
:100150009F0100089F0100089F0100089F010008FF
:100160009F0100089F0100089F0100089F010008EF
:10017000DFF80CD000F0DEFA0048004739400008F4
:10018000880C00200648804706480047FEE7FEE747
:10019000FEE7FEE7FEE7FEE7FEE7FEE7FEE7FEE737
:1001A0002D2500087101000840EA01039B0703D0D8
:1001B00009E008C9121F08C0042AFAD203E011F8A6
:1001C000013B00F8013B521EF9D27047D2B201E068
:1001D00000F8012B491EFBD270470022F6E710B54C
:1001E00013460A4604461946FFF7F0FF204610BDA5
:1001F000034611F8012B00F8012B002AF9D118460B
:1002000070472DE9FE4F81EA030404F0004421F019
:10021000004100944FF0000B23F0004350EA01042A
:100220005ED052EA03045BD0C3F30A54C1F30A550B
:100230002C44A4F2F3340194A0FB0254C1F3130143
:1002400041F48011C3F3130343F4801301FB024410
:1002500000FB034E840A970A44EA815447EA835715
:10026000A4FB076802958D0A05FB07854FEA932CCE
:1002700004FB0C542705029D4FEA065847EA16373F
:10028000B5EB08056EEB070C870E920E47EA811757
:1002900042EA8312A7FB0201B6EB0B0164EB0004F8
:1002A0002B0D43EA0C335E1844EB1C50DA465146E2
:1002B000E7FB0201C5F313044FEA0B3343EA14537F
:1002C0004FEA0432019C43EA0603A4F10C040294B1
:1002D000009CCDE900B400F0F7F803B0BDE8F08F62
:1002E00000200146F9E72DE9F04D81EA030404F00E
:1002F000004B21F0004514464FF0000A23F0004166
:1003000050EA050220D054EA01021DD0C5F30A5775
:100310000246C5F31303C1F31300C1F30A5640F4B8
:10032000801543F48013A7EB0608101BD64608F28D
:10033000FD3873EB050002D308F1010801E09218C3
:100340005B41B8F1000F03DA00200146BDE8F08DF3
:1003500000204FF48011064684460EE0171B73EB15
:10036000050705D3121B63EB050306434CEA010C9A
:1003700049084FEA300092185B4150EA0107EDD17D
:1003800052EA030012D082EA040083EA050108431E
:1003900005D0101BAB4106D20122002306E000224B
:1003A0004FF0004302E06FF0010253101AEB060019
:1003B0004CEB085110EB0A0041EB0B01BDE8F04D8E
:1003C00000F073B80EB540F2334102910021CDE93F
:1003D00000110A460B4600F077F803B000BD00F0AC
:1003E000004230F000400AD0C10D01F56071C0F349
:1003F000160042EA0151C20840071143704700202D
:100400000146704701F0004330B421F0004150EA4A
:10041000010206D00A0DA2F56072C1F31301002A91
:1004200002DC30BC00207047440F44EAC104C10024
:10043000E01830BC00EBC250AFF300800029A8BF29
:100440007047401C490008BF20F00100704710B4FD
:10045000B0FA80FC00FA0CF050EA010404BF10BCB2
:10046000704749B1CCF1200421FA04F411FA0CF1DF
:1004700018BF012121430843A3EB0C01CB1D4FEA18
:1004800000614FEA102042BF002010BC704700EB13
:10049000C35010440029A4BF10BC7047401C490041
:1004A00008BF20F0010010BC704710B5141E73F196
:1004B000000408DA401C41F1000192185B411A4324
:1004C00001D120F0010010BD2DE9F04D92469B4670
:1004D00011B1B1FA81F202E0B0FA80F22032904616
:1004E00000F03AF904460F4640EA0A0041EA0B01DF
:1004F00053465A46084313D0114653EA010019D017
:10050000C8F14002504600F036F905460E46504606
:100510005946424600F020F9084305D0012004E086
:1005200020463946BDE8F08D0020054346EAE076D6
:100530002C4337430A986305E40AA0EB0800002225
:10054000FD0A44EA47540A3002D500200146E9E793
:10055000010510196941DDE9084500196941BDE847
:10056000F04DA2E72DE9FE4F804681EA0300C00F5F
:100570000C46009021F0004123F00045B8EB02004A
:10058000A94105D24046214690461C460B460246EC
:1005900023F00040104347D0270DC7F30A00C3F3F0
:1005A0000A510290401A019040286BDAC3F31300FD
:1005B00040F4801B0098924620B10023D2EB030A3E
:1005C00063EB0B0B01985946C0F14002504600F016
:1005D000C3F806460D4650465946019A00F0DBF82E
:1005E00010EB08006141002487EA115284EAE773A6
:1005F0001A4340D0009A62B3019A012A4FEA075287
:1006000015DC001B61EB02014FF0004202EA0752C9
:10061000CDE90042001C41F5801132462B46FFF720
:1006200053FF03B0BDE8F08F40462146F9E7001BB9
:1006300061EB0201001C41F5801300185B4120189A
:10064000A2F5001747EB030140EAD570B6196D41DA
:1006500011E06D084FEA360645EAC0754FEA0752C9
:10066000001B61EB0201001C41F5801149084FEAB3
:1006700030000019514132462B4603B0BDE8F04F1F
:10068000FFF713BF0098012240000023D0EB0202C5
:1006900063EBE073009821464FEAE074B8EB00008A
:1006A00061EB0401E9E783F000435BE781F000417F
:1006B00058E770B521F0004303430CD0C1F30A554D
:1006C0000024D5EB040564EB0403D617AD1AB3413F
:1006D00002DB0020014670BD201841EB025170BDC5
:1006E0000EB5C10F80EAE0700844CA07002140F24D
:1006F00033438DE80E000A460B46FFF7E5FE03B0D4
:1007000000BD000030B5041E71F1000404DB4FF0A1
:100710000044404264EB0101141E73F1000405DB48
:100720001C464FF00043524263EB0403994208BF5A
:10073000904230BD064C074D06E0E06840F00103F2
:1007400094E8070098471034AC42F6D3FFF714FD45
:10075000E850000808510008202A04DB203A00FA7B
:1007600002F1002070479140C2F1200320FA03F308
:10077000194390407047202A04DB203A21FA02F006
:100780000021704721FA02F3D040C2F120029140CB
:10079000084319467047202A06DBCB17203A41FA56
:1007A00002F043EAE07306E041FA02F3D040C2F1FE
:1007B000200291400843194670472DE9F04D00236F
:1007C0001A461B1A8A4103DB00200146BDE8F08D62
:1007D000C1F30A52C1F3130141F480154FF0000B2D
:1007E000D10702D100186D41521E0027044640F285
:1007F000FF11384601EB620A3E4680460246002061
:100800004FF48011FFF7B7FFC2197141BB1846EBD7
:100810000100B4EB030C75EB000C04D3E41A65EB98
:10082000000517460E46241908F101006D41804667
:100830003428E3DDF91946EB0600091BA84103D271
:100840004FF0FF32134601E0002213461BEB070076
:1008500046EB0A51BDE8F04DFFF727BE30B5041E48
:1008600071F1000404DB4FF00044404264EB0101ED
:10087000141E73F1000405DB1C464FF00043524286
:1008800063EB04038B4208BF824230BD70B58C1805
:1008900010F8015B15F0070301D110F8013B2A1194
:1008A00006D110F8012B03E010F8016B01F8016B81
:1008B0005B1EF9D12B0705D40023521E0DD401F87D
:1008C000013BFAE710F8013BCB1A921C03E013F846
:1008D000015B01F8015B521EF9D5A142D8D300207B
:1008E00070BD000010B501221021024803F0DCFAAF
:1008F00010BD00000008014010B500221021024880
:1009000003F0D2FA10BD00000008014000BFFEE76E
:100910007047000010B5022003F04CFA48B10220E5
:1009200003F042FA01F0CEFD18B101200149096837
:10093000884710BD8400002000BFFEE700BFFEE72F
:100940007047000010B52823084A0A21022001F050
:100950002FFD08B1012010BDEF223421022001F04B
:100960009DFD08B10120F6E70020F4E78D0000208E
:1009700070B505460621022000F02AFD06461DB985
:1009800006F0FE00441C01E006F0FE0422460621AB
:10099000022001F083FD08B1012070BD0020FCE7BA
:1009A0002DE9F0432DED0A8B8BB0064600F08BFA53
:1009B000044600F046FA804600F03BFA074600F095
:1009C0006BFA08EE900A00F051FA054628224F49CA
:1009D00001A8FFF7E9FB062F01DB092F05DD002049
:1009E0000BB0BDEC0A8BBDE8F0830120A04000EE07
:1009F000100AB8EEC00A01A800EB8700D0ED000A8B
:100A000080EE209A9FED428A072C30DAB8EE680A11
:100A1000F1EE090A30EE200A60EE099AF000A0EB30
:100A20008400243000EE100AF8EEC00AA4EB450062
:100A3000800000EE100AB8EE400A80EE801A11EE37
:100A4000109A4846FFF7CBFC41EC1C0BB0EE4C0A69
:100A5000F0EE6C0A01F0BCFDB0EE40BAF0EE60BA08
:100A600051EC1B0BFFF7CEFC08EE100A2FE0B8EE9E
:100A7000680AF1EE010A30EE200A60EE099AF000F1
:100A8000A0EB84002C3000EE100AF8EEC00AA4EBB4
:100A90004500800000EE100AB8EE400A80EE801A91
:100AA00011EE109A4846FFF79AFC41EC1C0BB0EE91
:100AB0004C0AF0EE6C0A01F08BFDB0EE40BAF0EE9D
:100AC00060BA51EC1B0BFFF79DFC08EE100A08F111
:100AD000040000EE100AB8EEC00A28EE000AB0EEDC
:100AE000408AB2EE000A38EE000AB0EE408A28EEE4
:100AF000090AB0EE408A39EE880ADFED060A20EED8
:100B000020AABDEECA0A10EE100A69E7F84F0008E5
:100B10000000000000007A442DE9F0410025002685
:100B200000271FE03F226C21002001F0B7FC6C2160
:100B3000002000F04DFC044604F07F0010B90020B6
:100B4000BDE8F081681CC5B2002607E0002701E07F
:100B5000781C87B2642FFBDB701C86B2B6F5966FEB
:100B6000F4DB00BF032DDDDB0120E9E770B50024D5
:100B70000025042000F012FC054645F0100529462A
:100B8000042001F067FC4948816A0A20884705F083
:100B9000EF052946042001F05DFC002000F0FEFB7B
:100BA000044604F07F042146002001F053FC3F4836
:100BB000816A0A20884744F080042146002001F021
:100BC00049FC3A48816A0A20884704F07F0421469C
:100BD000002001F03FFC3548816A0A208847002147
:100BE000022001F037FC08B1012070BD2F48816A56
:100BF0000A2088470121022001F02CFC08B10120C5
:100C0000F3E72A48816A0A2088470621032000F07A
:100C1000DFFB064646F0200632460621032001F09F
:100C20003DFC08B10120E0E72048816A0A2088479E
:100C30000221084601F00EFC08B10120D5E71B484F
:100C4000816A0A2088472F222621032001F026FCF2
:100C500008B10120C9E71548816A0A208847362172
:100C6000042001F0F7FB08B10120BEE70F48816ABC
:100C70000A2088470D49486880470321022001F077
:100C8000E9FB08B10120B0E70848416A0220884723
:100C90000421022001F0DEFB08B10120A5E7034892
:100CA000816A0A20884700209FE700000801002091
:100CB00010B53E21022000F08BFB044644F00804EE
:100CC00022463E21022001F0E9FB08B1012010BDBF
:100CD0000020FCE710B53E21022000F079FB04461D
:100CE00024F0080422463E21022001F0D7FB08B17F
:100CF000012010BD0020FCE7FEB506460C46154657
:100D00000020009064270190029020128DF80400CA
:100D1000E0B28DF805006806000E8DF8060002208E
:100D200001F008FB032201A9304601F01FFB00BFC0
:100D30006C21002000F04CFB00F0800000B104E0CA
:100D4000381EA7F101018FB2F2D100BF022001F0DD
:100D5000F1FA01226946304600F0DCFA9DF8000005
:100D6000FEBD30B58BB0282101A8FFF736FAFFF79A
:100D7000B1FF11240DE004F10D00C2B245F6A5212A
:100D80003B20FFF7B9FF04F10D0101AA5054601C8C
:100D9000C4B2142CEFDB1C2245F6A5213B20FFF743
:100DA000ABFF5A2840D1FD223D21022001F076FB05
:100DB0009DF8240028B19DF824204521002001F051
:100DC0006DFB0D2245F6A5213B20FFF795FF01287D
:100DD00011D11C21032000F0FBFA054605F0E005C7
:100DE0009DF8220000F01F0005432A461C21032025
:100DF00001F054FB12E00D2245F6A5213B20FFF740
:100E00007BFF02280AD19DF8220000F01F0040F06D
:100E1000C0052A461C21032001F040FB9DF8232039
:100E20001D21032001F03AFBFFF742FF00200BB029
:100E300030BD10B50D21032000F0CAFA0446200988
:100E400010BD70B5002400250D21032000F0C0FA6C
:100E50000546C5F34204204670BD10B56C21002044
:100E600000F0B6FA044604F07F0010BD10B5122160
:100E7000032000F0ADFA0446C4F3C00010BD10B565
:100E8000022000F08BFA10BD10B52E21012000F0D9
:100E90009FFA0446E00910BD70B51321032000F04D
:100EA00097FA04461421032000F092FA054644EA1A
:100EB000052070BD10B500247F21012000F088FAC4
:100EC00044B2204610BD10B50E21032000F080FA78
:100ED0000446200910BD00002DE9F04F2DED108BC8
:100EE00083B09FED3D0A8DED020A7421012000F0D0
:100EF0006FFA05467521012000F06AFA0646762150
:100F0000012000F065FA0746380440EA062040EA6E
:100F1000050B7121022000F05BFA8046722102204D
:100F200000F056FA81467321022000F051FA824601
:100F30004FEA0A4040EA092040EA08047C210120E7
:100F400000F046FA0009019004B901242046FFF799
:100F500039FA41EC1B0B0198FFF734FA41EC1F0BF7
:100F6000B0EE4F1AF0EE6F1A9FED1C0B01F038FE39
:100F7000B0EE40DAF0EE60DA5846FFF723FA41ECC3
:100F80001E0B53EC1D2BFFF7AEF941EC1C0B53EC81
:100F90001B2BFFF7A8F941EC1A0BB0EE4A0AF0EE52
:100FA0006A0A01F085FDB0EE409AF0EE609A9FED7E
:100FB0000D0B53EC102B51EC190BFFF722F941EC00
:100FC000180BFFF71FFA02909DED020A03B0BDEC6B
:100FD000108BBDE8F08F0000000000000000000052
:100FE00000000040000000000000244010B51B225B
:100FF0000321002001F052FA08B1012010BD762231
:101000000421002001F04AFA08B10120F6E701228C
:101010000621002001F042FA08B10120EEE721226A
:101020001521002001F03AFA08B10120E6E7D022AC
:101030003121002001F032FA08B10120DEE76622FA
:101040003621002001F02AFA08B10120D6E76B22F0
:101050003721002001F022FA08B10120CEE7CC228E
:101060003821002001F01AFA08B10120C6E7092250
:101070003921002001F012FA08B10120BEE7B422A4
:101080003C21002001F00AFA08B10120B6E7422213
:101090003E21002001F002FA08B10120AEE76A22E9
:1010A0004021002001F0FAF908B10120A6E706224C
:1010B0004121002001F0F2F908B101209EE7AA22A7
:1010C0004221002001F0EAF908B1012096E77722D9
:1010D0004821002001F0E2F908B101208EE77722D3
:1010E0004921002001F0DAF908B1012086E77722D2
:1010F0004A21002001F0D2F908B101207EE7052243
:101100004B21002001F0CAF908B1012076E7042242
:101110004F21002001F0C2F908B101206EE7D22270
:101120005021002001F0BAF908B1012066E78022C1
:101130005E21002001F0B2F908B101205EE71B2218
:101140000321012001F0AAF908B1012056E7762217
:101150000421012001F0A2F908B101204EE7082284
:101160000B21012001F09AF908B1012046E70A227B
:101170000F21012001F092F908B101203EE7002281
:101180001921012001F08AF908B1012036E7D022A7
:101190002F21012001F082F908B101202EE7DA2287
:1011A0004321012001F07AF908B1012026E71B2232
:1011B0000321022001F072F908B101201EE7762216
:1011C0000421022001F06AF908B1012016E7C022CB
:1011D0002C21022001F062F908B101200EE727223C
:1011E0002D21022001F05AF908B1012006E7092259
:1011F0002E21022001F052F908B10120FEE6002262
:101200002F21022001F04AF908B10120F6E6102250
:101210003021022001F042F908B10120EEE61B2244
:101220000321084601F03AF908B10120E6E67622EA
:101230000421032001F032F908B10120DEE60E227C
:101240000A21032001F02AF908B10120D6E6CF22B5
:101250000B21032001F022F908B10120CEE619226A
:101260000C21032001F01AF908B10120C6E69822EA
:101270000D21032001F012F908B10120BEE616226B
:101280001221032001F00AF908B10120B6E6142268
:101290001321032001F002F908B10120AEE6F42287
:1012A0001621032001F0FAF808B10120A6E6012278
:1012B0001721032001F0F2F808B101209EE68322F5
:1012C0001A21032001F0EAF808B1012096E6D9229C
:1012D0001F21032001F0E2F808B101208EE6202250
:1012E0002621032001F0DAF808B1012086E600206B
:1012F00084E670B505460C461CB9284600F0A3F8F4
:1013000070BD012C03D1284600F080F8F8E70120D9
:10131000F6E700002DE9F04105460E46174600208D
:1013200040EA450000F0FF080A49086A804709487A
:10133000816940468847002405E00648816900200D
:1013400088473055641CBC42F7DB0249C8698047B6
:10135000BDE8F081080100202DE9F0414FF00008C0
:101360000921032000F034F804460A21032000F08C
:101370002FF805460B21032000F02AF806460C2121
:10138000032000F025F80746380640EA064040EA08
:10139000052040EA04084046BDE8F08170B50446E7
:1013A00000250A49086A8047002242EA4402D0B276
:1013B000064A9169884705488169002088470546A3
:1013C0000249C8698047284670BD00000801002016
:1013D00070B505460C46284600F0ACFF08B1012068
:1013E00070BD2046FFF7DAFFFAE770B50546002426
:1013F0007D210120FFF7ECFF04462246294601200B
:10140000FFF788FFFFF788FB204670BD70B50546E3
:101410001026002411E00A2C07D204F17600C1B294
:101420000220FFF7D5FF285506E004F16C00C1B299
:101430000020FFF7CDFF2855641CB442EBD3FFF723
:101440006BFBF0B270BD70B505460826002407E0BE
:1014500004F17600C1B20220FFF7BAFF2855641CE0
:10146000B442F5D3FFF758FBF0B270BD10B50024BD
:101470000020FFF793FF044644F08004214600203B
:1014800000F0E8FF0020FFF789FF044604F07F0426
:101490002146002000F0DEFF0020FFF77FFF002044
:1014A00010BD70B505460C46E2B20C21012000F0DB
:1014B000F5FF08B1012070BD0521022000F0CAFF30
:1014C00008B10120F7E722462946012000F04EFF2F
:1014D0000020F0E72DE9F04104460D210320FFF73D
:1014E00077FF0646304664F31F1000F0FF084246BF
:1014F0000D21032000F0D2FF10B10120BDE8F081E2
:10150000FFF7E1FC07460B2F07D1062C01D0072C73
:1015100001D101250EE000250CE00C2F09D1062C8D
:1015200003D0072C01D0082C01D1012502E00025B1
:1015300000E00025284603F04DFA062C03D0072CC6
:1015400001D0082C10D13F210220FFF741FF0646B1
:1015500046F0020632463F21022000F09FFF08B10C
:101560000120CBE70020C9E73F210220FFF730FF31
:10157000064606F0FD0632463F21022000F08EFFAF
:1015800008B10120BAE70020B8E770B5054600248D
:101590000D210320FFF71CFF044624F00E0444EA4B
:1015A0004500C4B222460D21032000F077FF08B1A8
:1015B000012070BD0020FCE770B504460E21032019
:1015C000FFF706FF054605F0F70040EAC400C6B283
:1015D00032460E21032000F061FF08B1012070BDEA
:1015E0000020FCE770B5044624210320FFF7F0FE3D
:1015F000054605F0F70040EAC400C6B23246242191
:10160000032000F04BFF08B1012070BD0020FCE773
:101610002DE9F0472DED088B04469FEDFE0AB0EE54
:10162000408A00269FEDFB0AF0EE408AB146FA4858
:10163000844206D22823F94A0A21022000F0B8FE8B
:1016400005E02823F64A0A21022000F0B1FEF54801
:1016500084422CD3F448844229D81A224021002005
:1016600000F01CFF20B10120BDEC088BBDE8F08725
:101670004FF00009A000FEF7A5FE41EC1B0B9FED0B
:10168000EB0B53EC102BFEF7BCFD41EC1A0B9FED5E
:10169000E90B53EC102BFEF726FE41EC190BFEF77D
:1016A000B1FE08EE100A002000F0FFFBCFE2DE489A
:1016B000844229D9E148844226D82A2240210020A8
:1016C00000F0ECFE08B10120CEE74FF00009A000C9
:1016D000FEF778FE41EC1B0B9FEDD40B53EC102B67
:1016E000FEF78FFD41EC1A0B9FEDD20B53EC102B44
:1016F000FEF7F9FD41EC190BFEF784FE08EE100A27
:10170000002000F0D2FBA2E2CC48844229D9CC4888
:10171000844226D83A224021002000F0BFFE08B1C2
:101720000120A1E74FF00009A000FEF74BFE41ECBD
:101730001B0B9FEDBE0B53EC102BFEF762FD41EC33
:101740001A0B9FEDBC0B53EC102BFEF7CCFD41ECBC
:10175000190BFEF757FE08EE100A002000F0A5FB5B
:1017600075E2B748844229D9B648844226D84A222D
:101770004021002000F092FE08B1012074E74FF0F4
:101780000009A000FEF71EFE41EC1B0B9FEDA70B0E
:1017900053EC102BFEF735FD41EC1A0B9FEDA50B1A
:1017A00053EC102BFEF79FFD41EC190BFEF72AFEC0
:1017B00008EE100A002000F078FB48E2A1488442BD
:1017C00029D9A148844226D85A224021002000F07D
:1017D00065FE08B1012047E74FF00009A000FEF7C1
:1017E000F1FD41EC1B0B9FED910B53EC102BFEF721
:1017F00008FD41EC1A0B9FED8F0B53EC102BFEF7FD
:1018000072FD41EC190BFEF7FDFD08EE100A0020F9
:1018100000F04BFB1BE28C48844229D98B48844260
:1018200026D86A224021002000F038FE08B10120AD
:101830001AE74FF00009A000FEF7C4FD41EC1B0BB6
:101840009FED7A0B53EC102BFEF7DBFC41EC1A0BEF
:101850009FED780B53EC102BFEF745FD41EC190B77
:10186000FEF7D0FD08EE100A002000F01EFBEEE1AE
:101870007648844229D97648844226D87A22402163
:10188000002000F00BFE08B10120EDE64FF000094A
:10189000A000FEF797FD41EC1B0B9FED640B53EC92
:1018A000102BFEF7AEFC41EC1A0B9FED620B53ECD4
:1018B000102BFEF718FD41EC190BFEF7A3FD08EE07
:1018C000100A002000F0F1FAC1E16148844229D9F0
:1018D0006048844226D87A224021002000F0DEFDB4
:1018E00008B10120C0E64FF00009A000FEF76AFD34
:1018F00041EC1B0B9FED4D0B53EC102BFEF781FCC5
:1019000041EC1A0B9FED4B0B53EC102BFEF7EBFC4D
:1019100041EC190BFEF776FD08EE100A002000F0EE
:10192000C4FA94E14C48844229D34C48844226D8D6
:101930001A224021002000F0B1FD08B1012093E6F9
:101940004FF000096000FEF73DFD41EC1B0B9FEDE1
:10195000370B53EC102BFEF754FC41EC1A0B9FEDA8
:10196000350B53EC102BFEF7BEFC41EC190BFEF7C8
:1019700049FD08EE100A012000F097FA67E13748A8
:10198000844229D93648844226D82A224021002080
:1019900000F084FD08B1012066E64FF00009600008
:1019A000FEF710FD41EC1B0B9FED200B53EC102BB1
:1019B000FEF727FC41EC1A0B9FED1E0B53EC102B8E
:1019C000FEF791FC41EC190BFEF71CFD08EE100A26
:1019D000012000F06AFA3AE12148844254D92148B2
:1019E000844251D83A224021002000F057FD08B12E
:1019F000012039E64FF000096000FEF7E3FC41ECFE
:101A00001B0B9FED0A0B53EC102BFEF7FAFB41EC7E
:101A10001A0B29E0000000000008AF2FB5000020DD
:101A2000DD00002040CF2318C065BC180000000076
:101A30000000F03F0000000080847E418047A11933
:101A40004029861A4056B71B4083E81C40B0191E37
:101A50008028971F4037AD21809E473080CB78315A
:101A6000008F423380520C351FED0E0B53EC102BC0
:101A7000FEF739FC41EC190BFEF7C4FC08EE100A26
:101A8000012000F012FAE2E0A148844229D9A148DD
:101A9000844226D84A224021002000F0FFFC08B1F1
:101AA0000120E1E54FF000096000FEF78BFC41ECFE
:101AB0001B0B1FED220B53EC102BFEF7A2FB41EC8E
:101AC0001A0B1FED240B53EC102BFEF70CFC41EC12
:101AD000190BFEF797FC08EE100A012000F0E5F95B
:101AE000B5E08C48844229D98B48844226D85A22B2
:101AF0004021002000F0D2FC08B10120B4E54FF0F5
:101B000000096000FEF75EFC41EC1B0B1FED390B7A
:101B100053EC102BFEF775FB41EC1A0B1FED3B0B42
:101B200053EC102BFEF7DFFB41EC190BFEF76AFCC0
:101B300008EE100A012000F0B8F988E076488442E7
:101B400029D97648844226D86A224021002000F014
:101B5000A5FC08B1012087E54FF000096000FEF701
:101B600031FC41EC1B0B1FED4F0B53EC102BFEF720
:101B700048FB41EC1A0B1FED510B53EC102BFEF7F9
:101B8000B2FB41EC190BFEF73DFC08EE100A0120F8
:101B900000F08BF95BE06148844229D960488442B7
:101BA00026D87A224021002000F078FC08B10120DC
:101BB0005AE54FF000096000FEF704FC41EC1B0BF6
:101BC0001FED660B53EC102BFEF71BFB41EC1A0BC1
:101BD0001FED680B53EC102BFEF785FB41EC190B46
:101BE000FEF710FC08EE100A012000F05EF92EE06E
:101BF0004B48844229D94B48844226D87A22402136
:101C0000002000F04BFC08B101202DE54FF0000949
:101C10006000FEF7D7FB41EC1B0B1FED7C0B53EC78
:101C2000102BFEF7EEFA41EC1A0B1FED7E0B53EC76
:101C3000102BFEF758FB41EC190BFEF7E3FB08EE07
:101C4000100A012000F031F901E001200CE5BDEEA1
:101C5000C80A10EE106AA6F1140800EE106AB8EE79
:101C6000C00A38EE400AF0EE408A9FED2F0A68EE77
:101C7000800A09F10100400000EE100AB8EEC00A27
:101C800080EE801ABDEEC10A10EE105A08F0FF0275
:101C90001521032000F002FC08B10120E4E4EAB2BF
:101CA0001621032000F0FAFB08B10120DCE4C5F3A3
:101CB00003221721032000F0F1FB08B10120D3E437
:101CC000E7B23A460921032000F0E8FB08B1012001
:101CD000CAE4C4F307273A460A21032000F0DEFBDA
:101CE00008B10120C0E4C4F307473A460B210320A2
:101CF00000F0D4FB08B10120B6E4270E3A460C21CF
:101D0000032000F0CBFB08B10120ADE40020ABE4E0
:101D100080520C3580AC6E378006D1398060333C00
:101D200000512E3F007E5F400000C84470B504465D
:101D30000025082C12DA63210020FFF749FB054635
:101D40000120A0402843C5B22A466321002000F0AC
:101D5000A5FB08B1012070BD0020FCE76421002034
:101D6000FFF736FB0546A4F10800012101FA00F057
:101D70002843C5B22A466421002000F08FFB08B139
:101D80000120E8E70020E6E770B504460025082CAE
:101D900012DA65210020FFF71BFB05460120A04059
:101DA0002843C5B22A466521002000F077FB08B120
:101DB000012070BD0020FCE766210020FFF708FB32
:101DC0000546A4F10800012101FA00F02843C5B23C
:101DD0002A466621002000F061FB08B10120E8E7F7
:101DE0000020E6E770B504460E460025082C17DAF9
:101DF00067210020FFF7ECFA05461EB90120A0403C
:101E0000854303E00120A0402843C5B22A4667214C
:101E1000002000F043FB08B1012070BD0020FCE76A
:101E200068210020FFF7D4FA05462EB9A4F1080076
:101E3000012181408D4306E0A4F10800012101FA4F
:101E400000F02843C5B22A466821002000F026FB96
:101E500008B10120E1E70020DFE710B54F210020A5
:101E6000FFF7B6FA044644F0080422464F2100204A
:101E700000F014FB08B1012010BD0020FCE770B594
:101E8000044612210320FFF7A3FA054605F0F700E8
:101E900040EAC400C6B232461221032000F0FEFA26
:101EA00008B1012070BD0020FCE770B50546002494
:101EB0003D210020FFF78CFA044624F0700415B988
:101EC00044F0100402E0012D00D100BFE2B23D2138
:101ED000002000F0E3FA08B1012070BD0020FCE70B
:101EE00010B504462146022000F0B4FA08B10120E2
:101EF00010BD0020FCE770B5054606210320FFF762
:101F000067FA044624F003042C43224606210320EA
:101F100000F0C4FA08B1012070BD0020FCE72DE9F3
:101F2000F0410546052D01D30C2D02D90120BDE855
:101F3000F0810E210320FFF74BFA8046404665F3FF
:101F40001F10C7B23A460E21032000F0A7FA08B1CD
:101F50000120ECE7FEF76DFF04460B2D07D1062CA0
:101F600001D0072C01D101260EE000260CE00C2D3B
:101F700009D1062C03D0072C01D0082C01D1012651
:101F800002E0002600E00026304602F023FD00209B
:101F9000CDE770B5054606210320FFF719FA044680
:101FA00024F0040444EA8500C4B22246062103203A
:101FB00000F074FA08B1012070BD0020FCE70000B9
:101FC0002DE9F0470446012C00DA0124FFF7C4F99B
:101FD0000646A248864272D3A14886426FD8172C83
:101FE00000DD16241E210020FFF7F2F9054605F05A
:101FF000C000611E01EB41019A4A515C40EA0108B0
:1020000042461E21002000F049FA10B10120BDE82F
:10201000F0874B210020FFF7DBF9054605F0F001C2
:10202000601E00EB40008F4A1044407841EA2018BF
:1020300042464B21002000F031FA08B10120E6E7CA
:1020400022210320FFF7C4F9054605F0FE00611EBA
:1020500001EB4101834A1144497801F0010140EA52
:10206000010842462221032000F018FA08B101209D
:10207000CDE7601E00EB40007A4908448078702864
:102080000ED046210020FFF7A3F9054645F00408CD
:1020900042464621002000F001FA88B10120B6E74F
:1020A00046210020FFF794F9054605F0FB0842465B
:1020B0004621002000F0F2F910B10120A7E72DE041
:1020C000FEF708FE202245F6A5213B20FEF714FE70
:1020D0008146FEF7EDFDB9F1000F01D14FF008097F
:1020E000601E00EB40005F490844807800F00F005C
:1020F000A9EB0000C5B2601E00EB400008448078E8
:1021000000F0F00040EA050842464521002000F0BA
:10211000C5F908B101207AE7002078E752488642E5
:1021200004D35248864201D8022709E04F4886422C
:1021300004D34F48864201D8032701E0012066E717
:10214000162C00DD16241E210020FFF741F905465C
:10215000601E484901EB001010F8270005F0C0018F
:1021600040EA010842461E21002000F097F908B11C
:1021700001204CE74B210020FFF72AF90546601E9D
:102180003C4901EB001000EB8700407805F0F001BE
:1021900040EA010842464B21002000F07FF908B1D7
:1021A000012034E722210320FFF712F90546601EC3
:1021B000304901EB001000EB8700807805F0FE014C
:1021C00040EA010842462221032000F067F908B1E5
:1021D00001201CE7601E274901EB001000EB87007F
:1021E000C078FF2828D046210020FFF7F1F80546E7
:1021F00045F0040842464621002000F04FF908B19E
:10220000012004E745210020FFF7E2F80546601EA3
:10221000184901EB001000EB8700C07805F08F0132
:1022200041EA001000F0FF0842464521002000F07E
:1022300035F980B10120EAE646210020FFF7C8F811
:10224000054605F0FB0842464621002000F026F92D
:1022500008B10120DBE60020D9E6000040CF2318BA
:102260004037AD21B04F0008809E473080520C357A
:10227000007E5F40504E000810B50121022000F0A2
:10228000E9F808B1012010BD2948816A0A20884771
:1022900006210320FFF79CF8044644F02004224660
:1022A0000621032000F0FAF808B10120EBE72048EE
:1022B000816A0A2088470221084600F0CBF808B15D
:1022C0000120E0E71A48816A0A2088472F22262148
:1022D000032000F0E3F808B10120D4E71448816A34
:1022E0000A2088473621042000F0B4F808B1012004
:1022F000C9E70F48816A0A2088470D494868804726
:102300000321022000F0A6F808B10120BBE708482D
:10231000416A022088470421022000F09BF808B19E
:102320000120B0E70248816A0A2088470020AAE716
:102330000801002070B50446002500260020FFF7A4
:102340002DF8064606F0FC0040EA04052946002068
:1023500000F080F80020FFF721F800F00300A04211
:1023600001D1002070BD0120FCE700002DE9F04103
:1023700005460E461746012040EA450000F0FF08DA
:102380000A49086A8047094881694046884700240D
:1023900004E0305D054A91698847641CBC42F8DB63
:1023A0000249C8698047BDE8F081000008010020AB
:1023B0002DE9F043C1B081460E4617461D464846FA
:1023C000FFF7B8FF18B1012041B0BDE8F08301204C
:1023D00040EA46081E49086A804708F0FF001C4A88
:1023E00091698847002405E0385D194A916988475A
:1023F000601CC4B2AC42F7DB1549C8698047144978
:10240000086A8047002242EA4602D0B2104A916927
:102410008847002407E00E4881690020884701A909
:102420000855601CC4B2AC42F5DB0949C869804755
:10243000002408E001A8005D395D884201D0012038
:10244000C2E7601CC4B2AC42F4DB0020BCE7000071
:10245000080100202DE9F04105460C460026012028
:1024600040EA4500C7B20C49086A80470A488169BA
:102470003846884708488169204688470649C86920
:1024800080472846FEF78AFF0646A64202D1002072
:10249000BDE8F0810120FBE70801002070B5064689
:1024A0000C4615463046FFF745FF08B1012070BDC8
:1024B00029462046FFF7CEFF08B10120F7E70020AC
:1024C000F5E7704710B50221014801F0A3FD10BDEA
:1024D000000C014010B501229102024801F0E4FC19
:1024E00010BD0000000C014010B500224FF48061C7
:1024F000014801F0D9FC10BD000C014010B50122CB
:10250000D102024801F0D0FC10BD0000000C0140D7
:1025100010B500224FF40061014801F0C5FC10BD68
:10252000000C014070477047704700001848006871
:1025300040F47000164908601648006820F0010059
:10254000401C1449086000BF12480068C0F34000F6
:102550000028F9D00F48406820F003000D4948607A
:1025600000BF0C484068C0F381000028F9D1094839
:10257000006809490840074908600020486008636E
:102580004FF41F008860C803014980390860704714
:1025900088ED00E000100240FFFFF2FE00BFFEE702
:1025A00003B401984100009850EAC12018BF0420EC
:1025B0004A0D18BF40F0010040F2FF72B2EB515FCC
:1025C00008BF40F00200012808BF052002B0704794
:1025D0002DE9F0412DED020B9FED3D0B2DED028B12
:1025E0009FED3D8BDDE90254C4F30A50A0F2FF36A3
:1025F000142E37DA002E18DA53EC102B9DED020B57
:1026000051EC100BFDF7AEFF53EC182BFEF77AF8E8
:1026100057D2002CBCBF4FF00044002551DB54EAD8
:10262000050018BF2E4C1BD14BE02E4820FA06F7B0
:1026300004EA070028431FD053EC102B9DED020B3A
:1026400051EC100BFDF78EFF53EC182BFEF75AF8E8
:1026500037D2002C03DD4FF48010F0400444BC431B
:1026600000252EE0332E07DCA6F114004FF0FF31D9
:1026700021FA00F73D4206D19DED020BBDEC028B25
:1026800002B0BDE8F08153EC102B9DED020B51EC34
:10269000100BFEF70BF853EC182BFEF733F810D2A3
:1026A000002C0DDD142E08BF641C09D0C6F13400C7
:1026B000012101FA00F02844A84238BF641C0546F5
:1026C000BD43CDE902549DED020BD7E700000000A9
:1026D0009C7500883CE4377E00000000000000008C
:1026E0000000F03FFFFF0F0070B5D94B00242DED27
:1026F000020B2DED108BDDE91010984205DA20F069
:1027000000429A4201D809D141B19DED100BBDECB8
:10271000108B02B0BDE8704001F01EB9B0F5801F0B
:1027200026DA11430BD0002813DA012001F068F9F2
:10273000BDEC108B02B0BDE8704001F021B9022061
:1027400001F05EF901F0F0F851EC100B81F000415E
:102750009EE06FF035049FEDC00B53EC102B9DED08
:10276000100B51EC100BFDF74CFDCDE910010846A4
:1027700004EB2051C0F31304B948A1F2FF31204407
:1027800000F4801080F07F6282F04052224301EB1F
:1027900020559FEDB50B119253EC102B9DED100BB6
:1027A00051EC100BFDF77FFF41EC180BA01CC0F3A0
:1027B00013009FEDAFDB9FEDB0EBB14E7E440328DD
:1027C0006CD296ED000B51EC180B53EC102BFEF76E
:1027D00045F81DD1002D01BF96ED000BBDEC108B0F
:1027E00002B070BD2846FDF77BFF41EC180B53EC9F
:1027F0001D2BFDF706FD41EC190B53EC1E2B51EC84
:10280000180BFDF7FEFC53EC192BFDF7ABFE3FE078
:102810009FED9D0B51EC180B53EC102BFDF7F1FCC9
:102820009FED9B1B53EC112BFDF740FF41EC190B67
:1028300053EC182B51EC180BFDF7E3FC53EC192B60
:10284000FDF7DFFC41EC190B002D04BF53EC192BF5
:1028500051EC180B1AD02846FDF742FF41EC1A0B39
:1028600053EC1D2BFDF7CDFC53EC192BFDF71EFF90
:1028700053EC182BFDF717FF41EC180B53EC1E2BF4
:1028800051EC1A0BFDF7BDFC53EC182BFDF70BFFB9
:10289000BDEC108B02B041EC100B70BD9FED7E0BB8
:1028A00051EC180B53EC102BFDF75CFE41EC100BB8
:1028B00051EC180B53EC102BFDF715FD41EC190BE7
:1028C0002846FDF70DFF41EC1B0B53EC192B51EC87
:1028D000190BFDF796FC41EC1A0B714853EC1A2BBF
:1028E000261851EC1A0BFDF78CFC41EC1F0B6D48C0
:1028F000C4F1510404F5D724B0EE4F0AF0EE6F0A8C
:102900000321784400F094FF53EC1F2B51EC100B83
:10291000FDF777FC41EC1C0B6348B0EE4F0AF0EE7C
:102920006F0A0421784400F083FF53EC1A2B51EC1A
:10293000100BFDF766FC344353EC1C2BFDF712FE25
:1029400041EC1C0B002C4CDD9FED510B51EC180B96
:1029500053EC102BFDF755FC53EC182BFDF751FCF5
:1029600041EC1A0B55B353EC1D2B51EC1B0BFDF72F
:1029700048FC41EC1D0B53EC1C2B51EC1A0BFDF7E2
:10298000F1FD53EC192BFDF73CFC53EC1D2BFDF72F
:10299000E9FD53EC1A2BFDF789FE53EC182BFDF7DC
:1029A00082FE41EC180B53EC1E2B51EC1B0BFDF778
:1029B00028FC53EC182BFDF776FE69E753EC1C2B33
:1029C00051EC1A0BFDF7CEFD53EC192BFDF719FC5A
:1029D00053EC1A2BFDF76AFE53EC182BFDF766FE3D
:1029E00056E735B353EC1D2B51EC1B0BFDF709FCDF
:1029F00041EC1A0B53EC1C2B51EC180BFDF753FE5A
:102A000053EC192BFDF7FDFB53EC1A2BFDF74BFE96
:102A100053EC182BFDF747FE41EC180B53EC1E2B23
:102A200051EC1B0BFDF7EDFB53EC182BFDF73BFEB8
:102A30002EE753EC1C2B51EC180BFDF734FE53EC36
:102A4000192BFDF7DEFB53EC182BFDF72FFE1FE7CC
:102A50000000F07F00000000000000000000504374
:102A6000645F090000000000000000000000F03F6B
:102A7000763C7935EF39EA3D0000E0FE422EE63F34
:102A80002029000000000000555555555555D53FEB
:102A9000000000000000E03F0000000000000040D7
:102AA00086EBF9FFA2270000982700000000000035
:102AB00070B5414A00252DED020B2DED048BDDE9AB
:102AC0000404944205DA24F00041914201D809D16E
:102AD00040B19DED040BBDEC048B02B0BDE870402D
:102AE00000F03ABFB4F5801F26DA08430BD0002C63
:102AF00013DA012000F084FFBDEC048B02B0BDE8C6
:102B0000704000F03DBF022000F07AFF00F00CFFA3
:102B100051EC100B81F0004146E09FED290B6FF066
:102B2000350553EC102B9DED040B51EC100BFDF70C
:102B300068FBCDE904010C4605EB2450A0F2FF3000
:102B4000C10F40F2FF32521A62F31F540844FDF7DE
:102B5000C7FD05949DED040B41EC180B51EC100BD7
:102B600001F061FA9FED181B53EC112BFDF749FBA7
:102B70009FED170B41EC190B53EC102B51EC180B7C
:102B8000FDF73FFB53EC192BFDF7ECFC9FED120B0F
:102B900041EC190B53EC102B51EC180BFDF731FBEA
:102BA00053EC192BFDF7DEFCBDEC048B02B041ECBD
:102BB000100B70BD000000000000F07F000000005E
:102BC00000000000000050430EE526157BCBDB3FE4
:102BD000362BF111F3FE593D00609F501344D33F53
:102BE0002DE9F04D2DED040B2DED0E8B96B0DDE9AA
:102BF0002550279CDDF890A025F0004624F00048E1
:102C0000BAF1000F14BF0121002101EB4502FC497C
:102C100053184A1093422AD3002814BF01230023DB
:102C200003EB44030B44F7498B4220D358EA0001DD
:102C30009FEDF59B76D0DFF8D8B35D4503D1BAF1AF
:102C4000000F05D188E0BAF1000F08BF002100D0C5
:102C5000012101EB450111F5001F08D8002814BF20
:102C60000121002101EB440111F5001F0BD99DED5D
:102C7000261B9DED240B16B0BDEC0E8B04B0BDE8F9
:102C8000F04D00F073BE0027002DBCBFE149884520
:102C900021DAE1498845A8BF02271CDAC3451ADCBE
:102CA000DE4901EB2851142908DDC1F1340220FA74
:102CB00002F101FA02F282420DD108E058B9C1F1E5
:102CC000140228FA02F101FA02F2424503D101F09E
:102CD0000101C1F1020756EA0A0124D1002C22DACF
:102CE000002D18BF022F01D0012F0AD0022000F0C2
:102CF00087FE16B0BDEC0E8B04B0BDE8F04D00F0C1
:102D000013BE022000F07CFE00F00EFE51EC100B12
:102D100081F0004141EC100B16B0BDEC0E8B04B0FD
:102D2000BDE8F08D18E09FEDBEAB9FEDBF8B002896
:102D300071D1B848804522D105F1804010F580104E
:102D400008BFBAF1000F07D0B3450ADC002CA8BFBA
:102D50009DED260BE0DA0DE0B0EE490AF0EE690ACF
:102D6000DAE7002C06DA9DED260B51EC100B81F012
:102D700000416FE0AE48784490ED000BCCE7D845B9
:102D80004DD1002C48DA2EB186423AD1BAF1000F6B
:102D900042D126E0BAF1000F13D0022000F030FE3D
:102DA00000F0FEFD8DED020B9DED240B8DED000B73
:102DB00010EE900A039961F31E0003909DED020B43
:102DC000AAE78DED02AB9DED240B1AEE901A10EEE2
:102DD000900A8DED000B61F31E0003909DED020B38
:102DE0009AE78DED028B9DED240B18EE901A10EEF4
:102DF000900A8DED000B61F31E0003909DED020B18
:102E00008AE709DA9DED240B51EC190B53EC102BDA
:102E1000FDF769FA1EE020E09DED240B7CE7864279
:102E20001BDAB4F1804F0DD0A4F10050B0F1FF5087
:102E300013D1002D11DB9DED240B51EC100B01F093
:102E40000BFF07E09DED240B53EC102B51EC100B06
:102E500000F0C2BC41EC100B5EE79DED240B51EC81
:102E6000100B01F001F8BAF1000FCDE90E0142D1CB
:102E70009FED710B46B3A6F1E040B0F17F600CD03E
:102E80005E4538D1002D00DAA7B3022F0CBF012018
:102E90004FF0FF30FDF724FCDCE7002D01DD002CB6
:102EA0000DDA002D01DD002C1FDB002D16DA002CC1
:102EB00014DB012F08BF9FED620B3FF42DAFB0EE86
:102EC0004A0AF0EE6A0A27E7022F18BF002D0CD03D
:102ED000012F0AD1002DFFF61FAF06E0002DB8BF6D
:102EE000002C08DA012F3FF417AFB0EE480AF0EEDD
:102EF000680A11E71BE0012000EBE57050EA0701CA
:102F000015D0791EB0EE498AF0EE698A084308BFF1
:102F10009FED4D8B4E480025804570DD4D494E4854
:102F2000884514DDB0420DDB002C19DB2FE00120B9
:102F300000F066FD16B0BDEC0E8B04B0BDE8F04DA0
:102F400000F01EBDB34502DC002C09DC1FE0864208
:102F500002DA002C1BDA03E05E452BDD002C16DDC7
:102F6000022000F04DFD00F01BFD8DED020B53EC37
:102F70001A2B51EC180BFDF744F9CDE90001039928
:102F8000019861F31E0003909DED020BC4E6022040
:102F900000F036FD00F014FD10EE901A18EE900AC5
:102FA0008DED020B8DED008B61F31E0003909DED06
:102FB000020BB1E69DED0E0B53EC192B51EC100BEF
:102FC000FDF771FB9FED260BCDE9080153EC102BAB
:102FD0009DED080B51EC100BFDF713F99FED221B33
:102FE00053EC112BFDF762FB9DED081B53EC112BED
:102FF000FDF707F99FED1E1B53EC112B3CE08CE015
:10300000FFFF1F00FFFF0F00000000000000F03F67
:103010000000F03F0000F07F0000404301FCFFFF94
:10302000000000000000F07F000000000000000031
:103030006623000000000000000000000000008087
:10304000000000000000F0FF000000000000F0BFE2
:103050000000E0410000F043FFFFEF3F00000000F0
:10306000000000000000D03F555555555555D53F3F
:10307000000000000000E03FFDF718FB9DED080B8D
:1030800041EC1A0B53EC102B51EC100BFDF7B9F877
:1030900053EC1A2BFDF7B5F841EC1A0B9FEDFE0B24
:1030A00053EC102B9DED080B51EC100BFDF7A9F81C
:1030B00041EC1B0B9FEDFA0B51EC1A0B53EC102B50
:1030C000FDF79FF841EC1A0B9FEDF70B53EC102B1B
:1030D0009DED080B51EC100BFDF793F853EC1A2BF8
:1030E000FDF7E1FA41EC1A0B51EC1B0B53EC1A2BD8
:1030F000FDF738FA0690CDE906519DED060B53EC2D
:103100001B2B51EC100BFDF7CEFA53EC1A2BFDF7ED
:10311000CDFA41EC100B00F0A1B90020B6F5801FEC
:103120000EDA9FEDE30B53EC102B9DED0E0B51ECE3
:10313000100BFDF766F8CDE90E016FF034000E4676
:1031400000EB2650A0F2FF37C6F31300DA4940F037
:103150007F6646F040568842D8BF002408DDD74934
:103160008142C8BF012403DC0024A6F580167F1C21
:10317000D348784400EBC4000F9690ED00CB9DED52
:103180000E0B53EC1C2B51EC100BFDF78CFA9DED44
:103190000E0B41EC1B0B53EC1C2B51EC100BFDF7F1
:1031A000E1F941EC100B51EC190B53EC102BFDF72E
:1031B0009AF841EC1D0B51EC1B0B53EC1D2BFDF74A
:1031C00020F841EC1A0BBF488DED10AB78441095F8
:1031D00090ED000B4FF0005040EA660000EB844099
:1031E0008DED080B00F5002009909DED080B53ECC8
:1031F0001C2B51EC100BFDF756FA9DED0E1B53ECFA
:10320000112BFDF753FA41EC100B53EC102B9DEDF5
:10321000100B51EC100BFCF7F4FF9DED080B41EC8B
:103220001C0B53EC102B9DED100B51EC100BFCF70D
:10323000E8FF53EC1B2BFDF739FA53EC1C2BFDF781
:1032400032FA53EC1D2BFCF7DCFF41EC1C0B53EC6A
:103250001A2B51EC1A0BFCF7D4FF41EC1B0B9A48CC
:103260000621B0EE4B0AF0EE6B0A784400F0E0FA6B
:10327000B0EE401AF0EE601AB0EE41DAF0EE61DA2C
:1032800053EC1B2B51EC1B0BFCF7BBFF53EC1D2B22
:10329000FCF7B7FF9DED100B41EC1B0B53EC1A2B09
:1032A00051EC100BFDF75EF953EC1C2BFCF7A9FF5A
:1032B00053EC1B2BFDF756F99DED100B41EC1B0B4E
:1032C00053EC102B51EC100BFCF79BFF41EC1D0B4A
:1032D0009FED7FEB53EC1E2BFDF744F953EC1B2BBA
:1032E000FDF740F90890CDE908519DED080B53EC2E
:1032F0001E2B51EC100BFDF7D6F953EC1D2BFDF7EF
:10330000D2F953EC1B2BFDF7D1F99DED080B41ECE5
:103310001D0B53EC102B9DED100B51EC100BFCF71B
:1033200070FF41EC1B0B53EC1A2B51EC1D0BFCF7FF
:1033300068FF9DED080B41EC1A0B53EC102B51EC80
:103340001C0BFCF75EFF53EC1A2BFDF70BF941EC5D
:103350001A0B51EC1B0B53EC1A2BFDF703F90C90D5
:10336000CDE90C519DED0C0B53EC1B2B51EC100BCC
:10337000FDF799F953EC1A2BFDF798F941EC1B0B6B
:103380009FED550B53EC102B9DED0C0B51EC100BDE
:10339000FCF737FF41EC1A0B9FED510B51EC1B0B67
:1033A00053EC102BFCF72DFF41EC1B0B9FED4E0B4C
:1033B00053EC102B9DED0C0B51EC100BFCF721FF87
:1033C00053EC1B2BFDF7CEF841EC100B484878442A
:1033D00000EBC40090ED001B51EC100B53EC112BD3
:1033E000FDF7C0F841EC1B0B3846FDF779F9CDE944
:1033F000080153EC1B2B51EC1A0BFDF7B3F841EC11
:10340000100B3C48784400EBC40090ED00CB51EC2D
:10341000100B53EC1C2BFDF7A5F89DED081B53EC8E
:10342000112BFDF79FF80690CDE906519DED080B95
:1034300053EC102B9DED060B51EC100BFDF733F9FF
:1034400053EC1C2BFDF72FF953EC1A2BFDF72BF93E
:1034500053EC1B2BFDF72AF941EC100B9DED261BBD
:1034600053EC102B8DED001B00959DED260B51ECC0
:10347000100BFCF7C6FE9DED000B41EC1A0B53EC54
:10348000102B9DED260B51EC100BFDF70CF99DED6B
:10349000061B53EC112B2FE0000000604715F73F8F
:1034A000FE822B654715F73F44DF5DF80BAE543EB7
:1034B00000000000000040438E9803007AB60B0025
:1034C000AA1E0000101F0000E21D00000000000006
:1034D0000000000000000840000000E009C7EE3FC7
:1034E000FD033ADC09C7EE3FF5015B14E02F3EBE59
:1034F0006E1C0000281C0000FCF783FE53EC1A2B06
:10350000FDF730F89DED060B41EC1A0B53EC102B38
:103510009DED000B51EC100BFCF773FECDE90C0197
:103520009DED0C0B51EC1A0B53EC102BFDF71AF818
:10353000CDE902010C46AA498C422FDB611A0843EF
:1035400018D19DED0C0B53EC102B9DED020B51ECA3
:10355000100BFDF7A8F841EC1B0B9FEDA30B51ECF2
:103560001A0B53EC102BFCF7FDFF53EC1B2BFDF754
:10357000C9F82DD2022000F043FA00F011FA10EE43
:10358000901A18EE900A8DED020B8DED008B61F311
:103590001E0003909DED020BFFF7BEBB944A24F082
:1035A0000041914214D39349214408437FF4EFAC86
:1035B0009DED0C0B53EC102B9DED020B51EC100B01
:1035C000FDF771F853EC1A2BFDF79CF87FF6DFAC92
:1035D00024F000408849894A002601EB20518242AC
:1035E0002BDA481C4FF4801121FA00F02044844A61
:1035F000C0F30A517A44A1F2FF3192ED000B814AE7
:103600008DED080BCA4020EA0202C0F3130040F41B
:103610008010C1F1140120FA01F60992002CB8BF04
:1036200076429DED080B53EC102B9DED0C0B51ECED
:10363000100BFDF738F8CDE90C019DED0C0B51ECAA
:103640001A0B53EC102BFCF78DFF9FED6F0B0890BE
:10365000CDE9085153EC102B9DED080B51EC100BEC
:10366000FCF7CFFD41EC1B0B9FED690B53EC102BCE
:103670009DED080B51EC100BFCF7C3FD9DED0C0B01
:1036800041EC1C0B53EC102B9DED080B51EC100B77
:10369000FDF709F853EC1A2BFDF708F89FED5E1BB8
:1036A00053EC112BFCF7ADFD53EC1C2BFCF75AFF30
:1036B00041EC1A0B51EC1B0B53EC1A2BFCF752FF8D
:1036C000CDE902019DED020B53EC1B2B51EC100BCD
:1036D000FCF7E9FF53EC1A2BFCF7E8FF9DED020B1A
:1036E00041EC1A0B53EC102B51EC100BFCF789FD3D
:1036F000CDE908014A489DED080B0521784400F00A
:1037000097F89DED081B51EC100B53EC112BFCF7B7
:1037100078FD9DED021B53EC112BFCF7C7FFCDE9A3
:1037200006019DED020B53EC1A2B51EC100BFCF72C
:1037300068FD53EC1A2BFCF715FF9FED3B0B41EC9A
:103740001A0B53EC102B9DED060B51EC100BFCF7F4
:10375000AAFF9DED060B41EC1B0B53EC102B9DEDCE
:10376000020B51EC100BFCF74CFD53EC1B2BFCF740
:10377000BAFD53EC1A2BFCF796FF9DED021B53ECA0
:10378000112BFCF790FF53EC192BFCF78FFFCDE9C1
:10379000020101EB065001150029C8BF039015DC9A
:1037A0009DED020B324651EC100BFCF782FFFEF749
:1037B000F7FE042808BF00F003F932469DED020B26
:1037C00051EC100BFCF775FFCDE902019DED020BEA
:1037D00051EC180B53EC102BFCF713FDFFF73ABB21
:1037E0000000904000000000FE822B654715973CCA
:1037F00000CC904000346F3F01FCFFFF0000E03F31
:10380000E81A0000FFFF0F0000000000432EE63F13
:10381000396CA80C615C20BEEF39FAFE422EE63FFF
:1038200080190000000000000000000000000040BF
:1038300070B504462DED028B4D1E00EBC500B0EEB9
:10384000408AF0EE608A90ED000B35F0060017D04C
:1038500053EC182B51EC100BFCF7D3FC41EC100B84
:103860006D1E04EBC50090ED001B51EC100B53ECEA
:10387000112BFCF777FE41EC100B35F00600E7D179
:10388000022D36D0042D1CD0062D1CBFBDEC028BA2
:1038900070BD53EC182B51EC100BFCF7B2FC94EDFF
:1038A0000A1B53EC112BFCF75DFE53EC182BFCF7B5
:1038B000A8FC94ED081B53EC112BFCF753FE41ECD4
:1038C000100B53EC182B51EC100BFCF79AFC94EDF9
:1038D000061B53EC112BFCF745FE53EC182BFCF7A1
:1038E00090FC94ED040B53EC102BFCF73BFE41ECE9
:1038F000100B53EC182B51EC100BFCF782FC94EDE1
:10390000021B53EC112BFCF72DFE53EC182BFCF78C
:1039100078FC94ED001B53EC112BFCF723FEBDEC5F
:10392000028B41EC100B70BD9FED070B10B553ECF3
:10393000102B9FED070B51EC100BFCF7D4FC41EC66
:10394000100B10BD0000000000000000000000008F
:10395000000000000000F03F10B553EC102B51ECBC
:10396000100BFCF7FFFD41EC100B10BD10B553EC34
:10397000112B51EC100BFCF7F5FD41EC100B10BDB9
:103980009FED050B10B553EC102B51EC100BFCF711
:10399000AAFC41EC100B10BD00000000000000006C
:1039A0009FED050B10B553EC102B51EC100BFCF7F1
:1039B00028FC41EC100B10BD00000000000000705E
:1039C0009FED050B10B553EC102B51EC100BFCF7D1
:1039D00018FC41EC100B10BD0000000000000010AE
:1039E00002E008C8121F08C1002AFAD170477047C8
:1039F000002001E001C1121F002AFBD17047000026
:103A000001490860704700004001002010B500F037
:103A100045F910BD0349496860F30711014A516037
:103A200070470000001002400349496860F30A2112
:103A3000014A516070470000001002400349496884
:103A400060F3CD21014A5160704700000010024030
:103A5000012807D10749496D21F030013031054A6D
:103A6000516505E00349496D21F03001014A516576
:103A70007047000000100240052827D2DFE800F060
:103A8000030A11181F00134A126861F30002114B58
:103A90001A601CE00F4A126861F310420D4B1A6065
:103AA00015E00C4A126861F318620A4B1A600EE0C6
:103AB000084A126A61F30002064B1A6207E0054ADF
:103AC000526A61F30002034B5A6200E000BF00BF7C
:103AD000704700000010024010B501460020094B5D
:103AE00003EB1142126801F01F040123A3401A40A6
:103AF00001F01F040123A3409A4200D000E00120FE
:103B000010BD00000010024030B50024002500E088
:103B1000641C1120FFF7E0FF012802D0B4F5405FDC
:103B2000F6D31120FFF7D8FF012801D0002500E0CF
:103B30000125284630BD000010B501290DD10E4BDE
:103B400003EB1042126800F01F040123A3401A4344
:103B5000094C04EB10431A600CE0074B03EB1042D6
:103B6000126800F01F040123A3409A43024C04EBA7
:103B700010431A6010BD00000010024010B568B973
:103B80001C4B5B6823F480331A4C636023461B6B29
:103B900023F0007303F10073236317E0154B5B6898
:103BA00023F4803303F58033124C6360012805D180
:103BB00023465B6823F40033636007E00D4B5B68CA
:103BC00023F4003303F500330A4C6360094B5B6850
:103BD00061F39543074C63600C09064B5B6864F323
:103BE0005E73044C636023465B6862F3DF7363605B
:103BF00010BD0000001002401348006820F00100D2
:103C0000401C1149086000BF0F480068C0F3400025
:103C10000028F9D00C48406820F003000A494860A9
:103C200000BF09484068C0F381000028F9D1064868
:103C3000006806490840044908600020486008639D
:103C40004FF41F008860704700100240FFFFF2FE33
:103C50000D49496860F301010B4A516000BF00BF84
:103C600000BF00BF00BF00BF00BF00BF00BF00BF5C
:103C700000BF00BF00BF00BF00BF00BF00BF00BF4C
:103C800000BF00BF704700000010024002484068BB
:103C9000C0F38100704700000010024010B50420FE
:103CA00001F0BAF8074800680749B0FBF1F007498E
:103CB0000860084600684FF47A7148430449086078
:103CC00010BD00003400002040420F0024000020FE
:103CD00028000020002131E032280ADD194A12684C
:103CE00032235A434FF0E0235A61A0F1320290B2DE
:103CF00006E0144A126842434FF0E0235A61002064
:103D000000224FF0E0239A611A46126942F0010244
:103D10001A6100BF4FF0E022116901F001021AB1EF
:103D200001F48032002AF5D04FF0E022126922F02F
:103D300001024FF0E0231A6100229A610028CBD1E2
:103D4000704700002800002001460020114A126838
:103D50004A434FF0E0235A6100229A611A461269E1
:103D600042F001021A6100BF4FF0E022106900F03A
:103D700001021AB100F48032002AF5D04FF0E0229F
:103D8000126922F001024FF0E0231A6100229A61C9
:103D90007047000024000020002141724160012191
:103DA000017201707047000001490860704700000F
:103DB00014040140014600200022044B1B6803EA62
:103DC00001020AB1012000E0002070471404014004
:103DD000014600204868234A12688243214B1A603A
:103DE0001A1D126882431B1D1A604A7A0AB30A78A8
:103DF0002AB91A1F126802431B1F1A6006E0194AEB
:103E0000121D12680243174B1B1D1A60154A083217
:103E100012688243134B08331A601A1D12688243DA
:103E20001B1D1A600A7A2AB91A1F126802431B1F47
:103E30001A6016E00A7A012A07D10A4A0C3212687F
:103E40000243084B0C331A600BE0064A0832126832
:103E50000243044B08331A601A1D126802431B1DEB
:103E60001A6070470004014082B0CDE9000121F0E2
:103E7000004001909DED000B02B051EC100B70471B
:103E80000246002109E0074800EB410090F90000DC
:103E9000904201DBC8B27047491C1729F3D31620A2
:103EA000F9E70000520000200AB1016100E0416121
:103EB00070474FF6FF71016000218171017104218B
:103EC00041710121C171704710B500228B071C0F91
:103ED0000F2303FA04F28B1033B1012B13D0022B02
:103EE00020D0032B3CD12CE01F4B9B6893431E4CEE
:103EF000A36023469B688C07240F00FA04F4234335
:103F0000194CA3602DE0184BDB689343164CE3601B
:103F10002346DB688C07240F00FA04F42343124C79
:103F2000E3601EE0104B1B6993430F4C2361234653
:103F30001B698C07240F00FA04F423430A4C236105
:103F40000FE0094B5B699343074C636123465B6950
:103F50008C07240F00FA04F42343034C636100E050
:103F600000BF00BF10BD000000000140F0B50A46D0
:103F70001588ABB29579032D01D100241AE095790B
:103F800065B9557905F00F045579182D01D10361F4
:103F900010E05579282D0DD143610BE0957905F09E
:103FA0000805167906F004063543D67906F00306AF
:103FB00045EA0604DDB2A5B1002110E001258D40DF
:103FC0001D405DB105688F000F26BE40B5430560FA
:103FD00005688E0004FA06F635430560491C082979
:103FE000ECD3FF2B15DD1B12002110E001258D40C5
:103FF0001D405DB145688F000F26BE40B54345604A
:1040000045688E0004FA06F635434560491C0829C8
:10401000ECD3F0BD0246002093680B408B4200D0E9
:1040200000E00120704710B541EC100BFEF75CFB7F
:1040300051EC100B10BD000000F045FE01211F489F
:10404000FFF77AFD01211D48401CFFF775FD012196
:104050001A48801CFFF770FD01211848C01CFFF7AB
:104060006BFDFFF7D3FC1649002000F055F9154809
:1040700000F07EFA0F2000F0B5FA03220721092094
:1040800000F088FA00F034FA16E00F48007888B99A
:104090004FF4FA7000F04CF801200B49087005202D
:1040A0000A4908730AA109480D30FCF7A1F807482E
:1040B00000F0B4FA00F05AF9E7E700000200180037
:1040C000994700080018DD19000000205802002060
:1040D00068656C6C6F00000070B50546002606E050
:1040E000601C84B2B4F5FA6F01DD002070BD0221BE
:1040F0000E4800F011FD0028F2D029460B4800F0D0
:1041000009FD002406E0601C84B2B4F5FA6F01DDFD
:104110000020EBE70121054800F0FEFC0028F2D06A
:10412000024800F0F3FCC6B23046DFE70030014041
:1041300010B50446A0B2FFF7CDFD10BD0121014A24
:1041400011707047800000201FB5044602A8FFF7D9
:10415000B0FE00208DF80C0001208DF80F00282003
:104160008DF80D0008208DF80E002020029002A985
:104170004548FFF7FBFE28208DF80D0000208DF844
:104180000E004020029002A93F48FFF7EFFE2820D2
:104190008DF80D0008208DF80E008020029002A9F5
:1041A0003948FFF7E3FE01213848FFF7C5FC6846B0
:1041B00000F09CFC00208DF8000001208DF801002B
:1041C00003208DF8020000208DF803008DF8040014
:1041D0008DF805008DF8060001208DF8070069466E
:1041E0002B4800F0A1FC0121294800F08AFC0120A5
:1041F0008DF80F0000208DF80C0010208DF80E00B7
:10420000029004208DF80D0002A91F48FFF7AEFEB2
:1042100001208DF80F0000208DF80C008DF80E00A5
:104220000220029018208DF80D0002A91948FFF70E
:104230009DFE01208DF80F0000208DF80C008DF8F8
:104240000E002020029018208DF80D0002A91248BF
:10425000FFF78CFE01208DF80F0000208DF80C0078
:104260008DF80E000420029018208DF80D0002A990
:104270000548FFF77BFEFCF735FBFEF753F900F02E
:104280000FF8064804601FBD000801400C0018002C
:1042900000300140000C014000100140840000206B
:1042A00000B585B06846FFF704FE01208DF80700D1
:1042B00000208DF804008DF80600022000901820E0
:1042C0008DF8050069461348FFF750FE01214FF4B1
:1042D000C010FFF731FC01210846FFF7F5FD02A8E9
:1042E000FFF75AFD01208DF8110000208DF808001D
:1042F0000220039000208DF8100002A8FFF768FD4F
:10430000032000F035FA00221146072000F0CCF916
:1043100005B000BD000C014070B506460C460F48C4
:10432000FFF712FF002500F0F3FA05460DB100BFBC
:10433000FEE700F02FFB0A48007800F024FB0A207B
:10434000FFF7F6FEFEF7E4F8FEF7CEF80CB10548ED
:104350000460E5200449086070BD00003D4100088C
:1043600081000020480000204C00002070B5ADF511
:10437000087D5A48006810B90DF5087D70BD584891
:10438000007800B9F8E700205549087055480078D2
:10439000022804D053480078032800D0ECE700F04E
:1043A0009DFA044604F0100068B100F09FFA05463B
:1043B000052000F04BFB29464B4800F0C7FA4A495C
:1043C000FF39A1F8190104F00800E8B300F096FAEB
:1043D00010EE100A4449FF39C1F8200500F08AFAAE
:1043E0004149FF3981F81F05022000F02FFB3E48AC
:1043F000FF3800F0B3FA3C49FF39A1F81B01002057
:1044000000F024FB39480068F0B13748FF3890F9D4
:104410001F05ADF814013448FF3890F81B018DF8E2
:1044200020013148FF38B0F81B2101460DF2211060
:10443000FBF7BAFE4FF4847246A96846FBF7B4FE58
:1044400000202A4E43A900E002E00EC93668B047BA
:1044500004F0040020B1042000F0F8FA00F0FBF9A9
:1044600004F00200E0B100F0F7FA032000F0EEFAE9
:1044700000F0F1F9002000F0E9FAFEF749F8FEF744
:1044800033F81A48006858B14FF4847246A9684658
:10449000FBF78AFE0120154E43A90EC93668B047C6
:1044A00004F00100B8B1012000F0DAFA00F0D3F90D
:1044B000FEF72EF8FEF718F80C48006858B14FF4D4
:1044C000847246A96846FBF76FFE0320074E43A996
:1044D0000EC93668B04700BF4EE700004C00002010
:1044E00080000020500000206304002048000020CD
:1044F00010B51848006800B910BDFEF709F8FDF7BF
:10450000E9FF00F0EFF9A8B900F0AAF91248006835
:1045100000F02EF8114890F9000000F063F8104800
:104520000278104801781048007800F033F80A202B
:10453000FFF7FEFD00F0D6F9012804D100F0BEFA25
:104540000A20FFF7F5FD00F0AFF9032007490870D6
:1045500000BFD1E74C0000203C00002038000020C4
:1045600046000020450000204400002050000020AC
:1045700010B504460548006800B910BD0448046041
:104580000168002000F02CFA00BFF6E74C00002084
:104590003C00002070B504460E4615460D480068E4
:1045A00000B970BD0C4804700C4806700C480570CA
:1045B0002946012000F014FA3146022000F010FADA
:1045C0002146032000F00CFA002000F003FA00BF9F
:1045D000E7E700004C0000204400002045000020D8
:1045E0004600002070B504460948006800B970BD57
:1045F0000848047090F90000FFF742FC064901EBFF
:10460000400045782946042000F0EAF900BFEEE7B3
:104610004C000020380000205200002010B5044655
:104620001A48006800B910BDFDF768FFFDF75CFF90
:1046300000F058F9A8B900F013F915480068FFF721
:1046400097FF144890F90000FFF7CCFF124802785A
:104650001248017812480078FFF79CFF0A20FFF704
:1046600067FD00F03FF9012804D100F027FA0A2085
:10467000FFF75EFD217B04F10802501D00F0F6F902
:1046800002200849087000BFCDE700004C00002060
:104690003C0000203800002046000020450000209B
:1046A00044000020500000202DE9F0470B4614463E
:1046B0004FF0000C00BF2C4A1268C2F302211D46C5
:1046C00026460A46C2F10709B9F1040F02D94FF094
:1046D000040901E0C2F10709C84602F10409B9F171
:1046E000070F02D24FF0000901E0A2F103094F4683
:1046F0004FF0010909FA08F9A9F1010909EA0509C8
:1047000009FA07F94FF0010A0AFA07FAAAF1010AB1
:104710000AEA060A49EA0A09CC4601466246002925
:1047200004DB15072E0E114D6E5407E015072F0EF2
:104730000D4D0C3501F00F06361FAF5500BF014679
:1047400000290DDB00BF00BF01F01F050122AA40B8
:104750004D09AD0005F1E025C5F8002100BF00BFFF
:1047600000BFBDE8F08700000CED00E000E400E0D1
:1047700000BF00F00702064B19684FF6FF0319400F
:10478000044B0B4343EA0221014B196000BF704701
:104790000CED00E00000FA050FB410B5044634B18A
:1047A000012C0DD0022C0ED0032C15D10EE04FF4AD
:1047B0008A7203A90B48FBF7F7FCFFF799FE0CE0A0
:1047C000FFF796FE09E0FFF793FE06E0FFF790FE85
:1047D00000200549087000E000BF00BF10BC5DF874
:1047E00014FB0000440100200000002010B500214F
:1047F0000846FDF7F7FA00210A20FDF7F3FA10BD8D
:1048000010B50A20FDF7C0FA0020FDF7BDFA0B2015
:10481000FDF78CFA00210A20FDF7E4FA0021084692
:10482000FDF7E0FA00210B20FDF7DCFA10BD10B512
:1048300000210846FDF7D6FA01210A20FDF7D2FA39
:1048400010BD10B500210A20FDF7CCFA012100208F
:10485000FDF7C8FA10BD10B5FCF75EF910BD0000F9
:1048600010B5FCF783F908B1012010BDFCF7BEFBC1
:1048700008B10120F9E7012000F076F808B1012025
:10488000F3E70249086880470020EEE708010020AE
:1048900010B50446A0B2FFF71DFA10BD10B50446CE
:1048A0002046FFF751FA10BD10B50420FDF718FBA4
:1048B00008B1012010BD0849C86880470220FDF7F3
:1048C0001AFB08B10120F5E70620FDF709FB08B146
:1048D0000120EFE70020EDE70801002010B5FCF70C
:1048E000BCFA10BD10B5FCF7CAFA10BD10B5FCF744
:1048F000CBFA10BD10B5FCF7DDFA10BD10B5FCF712
:10490000EBFA10BD10B504462046FCF749F810BD7F
:1049100010B5FCF72BF908B1012010BDFCF721FA06
:1049200008B10120F9E7FCF761FB08B10120F4E7C9
:10493000012000F019F808B10120EEE702490868EB
:1049400080470020E9E700000801002070B5044618
:104950000D4629462046FCF7CCFC70BD10B5044638
:104960002046FCF742FD10BD10B504462046FBF77B
:10497000FFFF08B1012010BDFBF7E4FF08B10120E3
:10498000F9E70020F7E710B504462046FCF72AFEB9
:1049900010BD000010B50420FDF7A2FA0C4900205C
:1049A00000F01EF80321012000F01AF80721022070
:1049B00000F016F80921032000F012F8012106206A
:1049C00000F00EF81621042000F00AF810BD0000D7
:1049D0000018DD1910B504462046FDF750FA10BD49
:1049E00070B505460C460420FDF77AFA072D29D24A
:1049F000DFE805F0040A10161C2822002046FCF708
:104A000007FE00F029F81EE0E0B2FCF7BEFD00F062
:104A100023F818E02046FCF75DFD00F01DF812E0D9
:104A20002046FDF77CFA00F017F80CE0E0B2FDF745
:104A3000C7FA00F011F806E02046FCF7BDFD00F0D3
:104A40000BF800E000BF00BF002070BD0149086006
:104A5000704700003401002010B5FCF707FD10BDC1
:104A600001490860704700003801002070B5064613
:104A70000C4615460420FDF733FA08B1012070BD3D
:104A8000FDF7EBF908B10120F9E70B498868804789
:104A90000020FDF77EFA08B10120F0E72046FFF77D
:104AA00031FF286021463046FCF7FBFC08B10120AD
:104AB000E5E70020E3E700000801002010B5FDF75E
:104AC000DBFB08B1012010BD0249086880470020C7
:104AD000F9E70000080100207047704710B5FBF7A8
:104AE00001FF10BD10B5FBF707FF10BD00210170DD
:104AF00041708170C1700171417181710121C17179
:104B00007047026861F38612026070470146C86808
:104B100080B27047C16070470246002093680B4026
:104B200003B900E001207047C26922F40062C2614B
:104B30000A7862B9026822F400420260026822F434
:104B400080420260026822F48062026036E00A78E5
:104B5000012A0ED1026822F400420260026822F4A7
:104B600080420260026822F4806202F58062026084
:104B700024E00A78022A0ED1026822F4004202F5EB
:104B800000420260026822F480420260026822F45D
:104B90008062026012E00A78032A0FD1026822F4D0
:104BA000004202F500420260026822F4804202F5EF
:104BB00080420260026822F480620260CB7902685F
:104BC00063F3492202604A78012A09D1CA79012A8D
:104BD00006D1026822F4807202F58072026003E05E
:104BE000026822F4807202604B78026863F38202EA
:104BF00002608A78072A0BDD426822F4807202F58F
:104C0000807242608A78036862F3C503036008E03B
:104C1000426822F4807242608B78026863F3C502B6
:104C20000260CB78026863F3C71202600B790268F6
:104C300063F3CB2202604B79026863F341020260A6
:104C40008B79026863F300020260704710B5044676
:104C50002046FFF741FA10BD00B52DED048B83B05F
:104C600041EC190BFBF7A9FD41EC180B18EE100AEB
:104C700018EE901A8DED008B002818BF0120084314
:104C800020F00040C0F17F6000F1E040C00F14D080
:104C900019EE101A19EE900A8DED009B002918BF2D
:104CA0000121084320F00040C0F17F6000F1E040A6
:104CB000C00F04BF0120FEF7A3FE51EC180B03B098
:104CC000BDEC048B00BD10B5FEF796FF0121084630
:104CD000FEF7D2FE00BFFEF717FF0028FBD001222F
:104CE0002F210220FEF74AFF01210220FEF7C4FE19
:104CF00000BF1920FEF7F0FE0128FAD10020FEF7D0
:104D000089FE0420FEF79AFE0420FEF78DFE0120A6
:104D1000FEF79EFE0220FEF79BFF00BFFEF7B6FFE8
:104D20000228FBD10020FEF793FE00F001F810BD31
:104D30002DE9F0470024002500260027A046FEF7B5
:104D4000A5FF8146B9F1000F06D0B9F1010F15D0CA
:104D5000B9F1020F3FD115E02948406DC0F3402062
:104D600040B12748006BC0F3406018B12548264980
:104D7000086002E025482449086030E023482249C1
:104D800008602CE01E484068C0F300461C4840689C
:104D9000C0F383441A484068C0F341750DB90F2C25
:104DA00003D12801401C044400E0A41C26B9184883
:104DB0006043154908600DE011484068C0F3404069
:104DC00020B1134860431049086003E00F48604376
:104DD0000D49086003E00D480B49086000BF00BFA3
:104DE00007484068C0F303170A4810F807800648D0
:104DF000006820FA08F004490860BDE8F087000068
:104E000000100240006CDC023400002000127A0026
:104E100000093D00404E0008042808D14FF0E02171
:104E2000096941F004014FF0E022116107E04FF001
:104E3000E021096921F004014FF0E022116170477F
:104E4000000000000000000001020304060708093A
:104E5000010B01FF010600FF010701FF010601FF31
:104E6000010B00FF01060000010B00FF010B01FF19
:104E7000030201FF03040100030001FF010B00FF17
:104E8000030801FF03000101030601FF030101FF05
:104E9000030B00FF030001FF030B00FF030701FFEB
:104EA000050001FF030B01FF050001FF030B00FFDD
:104EB000050301FF05010100050301FF050001FFD6
:104EC000050801FF07000100050B01FF050501FFB3
:104ED000050900FF07020100070001FF070001FFAD
:104EE000070201FF0D010100070201FF070401FF96
:104EF000070501FF0D020100090001FF070B01FF7B
:104F0000070B01FF0D040100090201FF090301FF66
:104F1000070B00FF0D060100090501FF0B0201FF51
:104F20000B0301FF0D0901000B0301FF0B0401FF3F
:104F30000B0501FF150401010B0601FF0D0401FF24
:104F4000150401FF150501010B0B01FF0D0701FF02
:104F5000150501FF150701010D0801FF150501FFEA
:104F6000150701FF15080101150601FF150701FFCF
:104F7000150100FF15010002150801FF150901FFC9
:104F8000150300FF15030002150200FF150300FFC3
:104F9000150500FF150500FF150500FF150500FFAD
:104FA000150600FF150600FF150600FF150600FF99
:104FB00001010003010103F03005018105A1810514
:104FC000F0810701810501800531800701800721FB
:104FD000800B11800B21800B41800B61800B918035
:104FE0000BB1800DB1800FB18011508015302015AC
:104FF000507015607000000000000000000000000C
:1050000000000000000000000000000000000000A0
:1050100000007A420000FA4200007A430000FA439E
:10502000000000000000F03F000000000000F83F1A
:1050300000000000000000000000004003B8E23F54
:10504000000000000000000006D0CF43EBFD4C3E06
:10505000033333333333E33FFFAB6FDBB66DDB3FFB
:105060004D268F515555D53F01411DA96074D13F43
:1050700065DBC9934A86CD3FEF4E454A287ECA3F3D
:105080003E5555555555C53F93BDBE166CC166BFBF
:105090002CDE25AF6A56113FF16BD2C541BDBBBEB8
:1050A000D0A4BE726937663E04FA97999999D93FA0
:1050B000AF788E1DC571CC3F9FC678D0099AC33F8B
:1050C000935555555555E53F599322942449D23F60
:1050D000DE03CB966446C73F44523EDF12F1C23F27
:1050E000000000000000000008510008000000203F
:1050F000440100008C080008B85100084401002059
:10510000440B0000F0390008516C100140041204F7
:105110001208322012047A1804C14201031B127AC9
:10512000D02FE601EF02FB03FD04FE05FF06020798
:1051300004080509070A080B090C0A0D0B0E0C0FD1
:105140000D100E110F12101311141215131614173F
:105150001206ABF8060408192614C0F91422D4F973
:105160002230D8F9303EDEF93E0EFF804F128038F3
:105170000128AD0980F3090418161406F01422C69C
:10518000F1223173F0313FDEF13F0EFFE03229288A
:1051900029D812481408DB4A1B0843081A2F0413A5
:1051A000ED471B08D910134D4C1B08DD081AE50408
:0851B0001A91181A9D04011068
:04000005080001717D
:00000001FF
